:020000020000FC
:1000000042C03AC040C03FC03EC017C03CC03BC029
:100010003AC039C038C037C036C035C034C0E199A5
:10002000FECF4EBB5DBBE29AE19A0895E199FECF07
:100030004EBBE09A3CB35DB30895DF93DFB7DF9327
:1000400030E033BF6AE06A95F1F734E033BFD2EBBA
:10005000D2BFD1E02D1B28F41D1B18F4002309F09A
:100060000A95DF91DFBFDF911895DF93DFB7DF934C
:10007000DF91DFBFDF911895DF93DFB7DF93DF916B
:10008000DFBFDF9118953FE53DBFBB98C39AB89A93
:10009000C09830E03ABD34E93EBD3CE93DBD32E0B8
:1000A00039BF33273FBB789441E0C0DF052F42E0E2
:1000B000BDDF152F43E0BADF252F322F3F3FA9F4D4
:1000C000312F3F3F91F4302F3F3F79F430E0032F41
:1000D000502F41E0A4DF36E4132F512F42E09FDF81
:1000E00030E5232F522F43E09ADF009371001093E5
:1000F00072002093730045E099DFC52ECC2011F0EB
:1001000034E901C03CE83EBD38ED30BF32EB32BFD0
:1001100034E033BFB3990FC00023F1F71123E1F7A7
:100120002223D1F7CC2011F03CE801C034E93EBDD8
:1001300000C00000FECF0FEF1FEF2FEFB39901C0FB
:1001400006C00D3FD9F71034C9F72F3DB9F7F89421
:10015000CC2011F03CE801C034E93EBD3FEF3C1932
:1001600045E0532F5CDF3FEF6FEF7FEF321B610BFA
:10017000700B41E0572F53DF42E0562F50DF43E032
:06018000532F4DDFD6CF26
:00000001FF
